******************************************************************************
                  TI ARM Linker PC v16.9.4                     
******************************************************************************
>> Linked Wed Dec 06 15:45:29 2017

OUTPUT FILE NAME:   <sensor_hub_testing_hub.out>
ENTRY POINT SYMBOL: "_c_int00"  address: 00002d1d


MEMORY CONFIGURATION

         name            origin    length      used     unused   attr    fill
----------------------  --------  ---------  --------  --------  ----  --------
  FLASH                 00000000   00040000  00003794  0003c86c  R  X
  SRAM                  20000000   00008000  00000ab5  0000754b  RW X


SEGMENT ALLOCATION MAP

run origin  load origin   length   init length attrs members
----------  ----------- ---------- ----------- ----- -------
00000000    00000000    00003798   00003798    r-x
  00000000    00000000    0000026c   0000026c    r-- .intvecs
  0000026c    0000026c    00003210   00003210    r-x .text
  00003480    00003480    000002d8   000002d8    r-- .const
  00003758    00003758    00000040   00000040    r-- .cinit
20000000    20000000    00000ab8   00000000    rw-
  20000000    20000000    0000067d   00000000    rw- .bss
  20000680    20000680    00000400   00000000    rw- .stack
  20000a80    20000a80    00000038   00000000    rw- .data


SECTION ALLOCATION MAP

 output                                  attributes/
section   page    origin      length       input sections
--------  ----  ----------  ----------   ----------------
.intvecs   0    00000000    0000026c     
                  00000000    0000026c     startup_ccs.obj (.intvecs)

.text      0    0000026c    00003210     
                  0000026c    00000588     rtsv7M4_T_le_v4SPD16_eabi.lib : e_powf.obj (.text)
                  000007f4    0000046c     sensor_hub_testing.obj (.text:main)
                  00000c60    0000023c     rtsv7M4_T_le_v4SPD16_eabi.lib : strtod.obj (.text)
                  00000e9c    000001f8     sensorlib.lib : bmp180.obj (.text:BMP180Callback)
                  00001094    000001ea     uartstdio.obj (.text:UARTvprintf)
                  0000127e    000001b6     rtsv7M4_T_le_v4SPD16_eabi.lib : fd_add_t2.obj (.text)
                  00001434    00000194     sensorlib.lib : mpu9150.obj (.text:MPU9150Callback)
                  000015c8    00000160     uartstdio.obj (.text:UARTStdioIntHandler)
                  00001728    00000136     rtsv7M4_T_le_v4SPD16_eabi.lib : fd_div_t2.obj (.text)
                  0000185e    00000132     driverlib.lib : gpio.obj (.text:GPIOPadConfigSet)
                  00001990    00000110                   : sysctl.obj (.text:SysCtlClockGet)
                  00001aa0    00000104     rgb.obj (.text:RGBInit)
                  00001ba4    000000fc     rtsv7M4_T_le_v4SPD16_eabi.lib : fd_mul_t2.obj (.text)
                  00001ca0    000000f2     sensorlib.lib : i2cm_drv.obj (.text:I2CMIntHandler)
                  00001d92    00000002     startup_ccs.obj (.text:FaultISR)
                  00001d94    000000d4     rtsv7M4_T_le_v4SPD16_eabi.lib : s_scalbnf.obj (.text)
                  00001e68    000000c0     rgb.obj (.text:RGBEnable)
                  00001f28    000000b0     uartstdio.obj (.text:UARTStdioConfig)
                  00001fd8    000000a8     uartstdio.obj (.text:UARTwrite)
                  00002080    000000a8     sensor_hub_testing.obj (.text:comenzi)
                  00002128    0000009c     rtsv7M4_T_le_v4SPD16_eabi.lib : memcpy_t2.obj (.text)
                  000021c4    00000098     sensorlib.lib : i2cm_drv.obj (.text:I2CMStateIdle)
                  0000225c    00000090     rgb.obj (.text:RGBColorSet)
                  000022ec    0000008c     uartstdio.obj (.text:UARTPrimeTransmit)
                  00002378    00000088     sensorlib.lib : i2cm_drv.obj (.text:I2CMCommand)
                  00002400    00000086     rtsv7M4_T_le_v4SPD16_eabi.lib : fd_cmp_t2.obj (.text:__aeabi_cdcmple)
                  00002486    00000002     startup_ccs.obj (.text:IntDefaultHandler)
                  00002488    00000084     sensorlib.lib : bmp180.obj (.text:BMP180DataTemperatureGetFloat)
                  0000250c    0000007c                   : mpu9150.obj (.text:MPU9150DataAccelGetFloat)
                  00002588    0000007a     rtsv7M4_T_le_v4SPD16_eabi.lib : memset_t2.obj (.text)
                  00002602    00000002     startup_ccs.obj (.text:NmiSR)
                  00002604    00000078     sensorlib.lib : i2cm_drv.obj (.text:I2CMReadModifyWrite8)
                  0000267c    00000078     rgb.obj (.text:RGBBlinkRateSet)
                  000026f4    00000070     rtsv7M4_T_le_v4SPD16_eabi.lib : autoinit.obj (.text)
                  00002764    0000006e                                   : fd_tos_t2.obj (.text)
                  000027d2    00000002                                   : i_div0.obj (.text)
                  000027d4    0000006c     sensorlib.lib : mpu9150.obj (.text:MPU9150Init)
                  00002840    00000068     driverlib.lib : interrupt.obj (.text:IntDisable)
                  000028a8    00000068                   : interrupt.obj (.text:IntEnable)
                  00002910    00000068     rgb.obj (.text:RGBDisable)
                  00002978    00000068     rtsv7M4_T_le_v4SPD16_eabi.lib : copy_decompress_lzss.obj (.text:decompress:lzss)
                  000029e0    00000064     sensor_hub_testing.obj (.text:ConfigureUART)
                  00002a44    00000064     driverlib.lib : interrupt.obj (.text:IntIsEnabled)
                  00002aa8    00000060     sensorlib.lib : i2cm_drv.obj (.text:I2CMReadModifyWrite8Callback)
                  00002b08    00000060                   : mpu9150.obj (.text:MPU9150DataRead)
                  00002b68    0000005e                   : i2cm_drv.obj (.text:I2CMStateWritePause)
                  00002bc6    00000002     rtsv7M4_T_le_v4SPD16_eabi.lib : mpu_init.obj (.text)
                  00002bc8    00000058     sensorlib.lib : bmp180.obj (.text:BMP180DataRead)
                  00002c20    00000054                   : bmp180.obj (.text:BMP180Init)
                  00002c74    00000054                   : mpu9150.obj (.text:MPU9150ReadModifyWrite)
                  00002cc8    00000054     uartstdio.obj (.text:UARTgets)
                  00002d1c    00000054     rtsv7M4_T_le_v4SPD16_eabi.lib : boot.obj (.text)
                  00002d70    00000054                                   : exit.obj (.text)
                  00002dc4    00000050     sensorlib.lib : i2cm_drv.obj (.text:I2CMStateWriteFinal)
                  00002e14    00000050     rtsv7M4_T_le_v4SPD16_eabi.lib : fs_toull_t2.obj (.text)
                  00002e64    0000004c     driverlib.lib : i2c.obj (.text:I2CMasterInitExpClk)
                  00002eb0    0000004c     rtsv7M4_T_le_v4SPD16_eabi.lib : cpy_tbl.obj (.text)
                  00002efc    0000004a     sensorlib.lib : i2cm_drv.obj (.text:I2CMStateReadNext)
                  00002f46    00000048                   : i2cm_drv.obj (.text:I2CMStateWriteNext)
                  00002f8e    00000044                   : i2cm_drv.obj (.text:I2CMStateCallback)
                  00002fd2    00000002     rtsv7M4_T_le_v4SPD16_eabi.lib : startup.obj (.text)
                  00002fd4    00000044     uartstdio.obj (.text:UARTPeek)
                  00003018    00000042     sensorlib.lib : i2cm_drv.obj (.text:I2CMStateReadFinal)
                  0000305a    00000040     rtsv7M4_T_le_v4SPD16_eabi.lib : u_divt2.obj (.text)
                  0000309a    0000003e     sensorlib.lib : i2cm_drv.obj (.text:I2CMStateReadPause)
                  000030d8    0000003c     uartstdio.obj (.text:UARTFlushTx)
                  00003114    00000038     rgb.obj (.text:RGBBlinkIntHandler)
                  0000314c    00000036     sensorlib.lib : mpu9150.obj (.text:MPU9150DataMagnetoGetRaw)
                  00003182    00000034                   : i2cm_drv.obj (.text:I2CMInit)
                  000031b6    00000002     --HOLE-- [fill = 0]
                  000031b8    00000030     sensor_hub_testing.obj (.text:SysTickIntHandler)
                  000031e8    0000002c     uartstdio.obj (.text:UARTFlushRx)
                  00003214    0000002a     driverlib.lib : gpio.obj (.text:GPIODirModeSet)
                  0000323e    0000002a     sensorlib.lib : i2cm_drv.obj (.text:I2CMStateReadFirst)
                  00003268    00000028     rtsv7M4_T_le_v4SPD16_eabi.lib : e_sqrtf.obj (.text)
                  00003290    00000022     driverlib.lib : pwm.obj (.text:PWMGenConfigure)
                  000032b2    00000020     sensorlib.lib : i2cm_drv.obj (.text:I2CMStateReadOne)
                  000032d2    0000001a                   : i2cm_drv.obj (.text:I2CMStateReadWait)
                  000032ec    0000001a     uartstdio.obj (.text:UARTprintf)
                  00003306    00000018     uartstdio.obj (.text:IsBufferFull)
                  0000331e    00000002     --HOLE-- [fill = 0]
                  00003320    00000018     rtsv7M4_T_le_v4SPD16_eabi.lib : args_main.obj (.text)
                  00003338    00000014     rgb.obj (.text:RGBIntensitySet)
                  0000334c    00000014     rtsv7M4_T_le_v4SPD16_eabi.lib : _lock.obj (.text)
                  00003360    00000014                                   : strcpy.obj (.text)
                  00003374    00000014                                   : strlen.obj (.text)
                  00003388    00000012     driverlib.lib : gpio.obj (.text:GPIOPinTypeI2CSCL)
                  0000339a    00000012     uartstdio.obj (.text:GetBufferCount)
                  000033ac    00000012     rtsv7M4_T_le_v4SPD16_eabi.lib : s_copysignf.obj (.text)
                  000033be    00000002     --HOLE-- [fill = 0]
                  000033c0    00000010     sensor_hub_testing.obj (.text:BMP180AppCallback)
                  000033d0    00000010     driverlib.lib : pwm.obj (.text:PWMGenPeriodSet)
                  000033e0    0000000e     uartstdio.obj (.text:IsBufferEmpty)
                  000033ee    0000000e     rtsv7M4_T_le_v4SPD16_eabi.lib : copy_decompress_none.obj (.text:decompress:none)
                  000033fc    0000000c     sensorlib.lib : bmp180.obj (.text:BMP180DataTemperatureGetRaw)
                  00003408    0000000c     sensor_hub_testing.obj (.text:BMP180I2CIntHandler)
                  00003414    0000000c     driverlib.lib : interrupt.obj (.text:IntTrigger)
                  00003420    0000000c     sensor_hub_testing.obj (.text:MPU9150Callback)
                  0000342c    0000000c     rtsv7M4_T_le_v4SPD16_eabi.lib : copy_zero_init.obj (.text:decompress:ZI)
                  00003438    0000000a     driverlib.lib : i2c.obj (.text:I2CMasterEnable)
                  00003442    00000008                   : i2c.obj (.text:I2CMasterIntClear)
                  0000344a    00000008                   : i2c.obj (.text:I2CMasterIntEnableEx)
                  00003452    00000008                   : i2c.obj (.text:I2CMasterSlaveAddrSet)
                  0000345a    00000006                   : gpio.obj (.text:GPIOPinWrite)
                  00003460    00000006     startup_ccs.obj (.text:ResetISR)
                  00003466    00000006     driverlib.lib : uart.obj (.text:UARTClockSourceSet)
                  0000346c    00000004                   : i2c.obj (.text:I2CMasterControl)
                  00003470    00000004                   : i2c.obj (.text:I2CMasterDataGet)
                  00003474    00000004                   : i2c.obj (.text:I2CMasterDataPut)
                  00003478    00000004     rtsv7M4_T_le_v4SPD16_eabi.lib : pre_init.obj (.text)

.const     0    00003480    000002d8     
                  00003480    00000101     rtsv7M4_T_le_v4SPD16_eabi.lib : ctype.obj (.const:.string:_ctypes_)
                  00003581    00000007     --HOLE-- [fill = 0]
                  00003588    00000098                                   : strtod.obj (.const:$O1$$)
                  00003620    00000070     driverlib.lib : interrupt.obj (.const)
                  00003690    0000006c                   : sysctl.obj (.const:g_pui32Xtals)
                  000036fc    00000020     sensorlib.lib : mpu9150.obj (.const)
                  0000371c    00000018     rtsv7M4_T_le_v4SPD16_eabi.lib : e_powf.obj (.const:$O1$$)
                  00003734    0000000c     uartstdio.obj (.const:g_ui32UARTBase)
                  00003740    0000000c     uartstdio.obj (.const:g_ui32UARTInt)
                  0000374c    0000000c     uartstdio.obj (.const:g_ui32UARTPeriph)

.cinit     0    00003758    00000040     
                  00003758    00000016     (.cinit..data.load) [load image, compression = lzss]
                  0000376e    00000002     --HOLE-- [fill = 0]
                  00003770    0000000c     (__TI_handler_table)
                  0000377c    00000004     --HOLE-- [fill = 0]
                  00003780    00000008     (.cinit..bss.load) [load image, compression = zero_init]
                  00003788    00000010     (__TI_cinit_table)

.init_array 
*          0    00000000    00000000     UNINITIALIZED

.bss       0    20000000    0000067d     UNINITIALIZED
                  20000000    00000400     uartstdio.obj (.bss:g_pcUARTTxBuffer)
                  20000400    00000124     (.common:g_sI2CInst)
                  20000524    00000080     uartstdio.obj (.bss:g_pcUARTRxBuffer)
                  200005a4    0000006c     (.common:sMPU9150)
                  20000610    00000044     (.common:g_sBMP180Inst)
                  20000654    0000000c     rgb.obj (.bss:g_ui32Colors)
                  20000660    0000000c     (.common:g_pui32Colors)
                  2000066c    00000008     uartstdio.obj (.bss)
                  20000674    00000004     rgb.obj (.bss)
                  20000678    00000004     (.common:g_vui8DataFlag)
                  2000067c    00000001     (.common:g_bMPU9150Done)

.stack     0    20000680    00000400     UNINITIALIZED
                  20000680    00000400     --HOLE--

.data      0    20000a80    00000038     UNINITIALIZED
                  20000a80    00000015     uartstdio.obj (.data)
                  20000a95    00000003     --HOLE--
                  20000a98    0000000c     rtsv7M4_T_le_v4SPD16_eabi.lib : exit.obj (.data:$O1$$)
                  20000aa4    00000008                                   : _lock.obj (.data:$O1$$)
                  20000aac    00000004     rgb.obj (.data)
                  20000ab0    00000004     rtsv7M4_T_le_v4SPD16_eabi.lib : errno.obj (.data)
                  20000ab4    00000004                                   : stkdepth_vars.obj (.data)

MODULE SUMMARY

       Module                     code    ro data   rw data
       ------                     ----    -------   -------
    .\
       sensor_hub_testing.obj     1488    0         485    
       startup_ccs.obj            12      620       0      
    +--+--------------------------+-------+---------+---------+
       Total:                     1500    620       485    
                                                           
    .\drivers\
       rgb.obj                    896     0         20     
    +--+--------------------------+-------+---------+---------+
       Total:                     896     0         20     
                                                           
    .\utils\
       uartstdio.obj              1664    36        1181   
    +--+--------------------------+-------+---------+---------+
       Total:                     1664    36        1181   
                                                           
    C:/ti/TivaWare_C_Series-2.1.4.178/driverlib/ccs/Debug/driverlib.lib
       interrupt.obj              320     112       0      
       sysctl.obj                 272     108       0      
       gpio.obj                   372     0         0      
       i2c.obj                    122     0         0      
       pwm.obj                    50      0         0      
       uart.obj                   6       0         0      
    +--+--------------------------+-------+---------+---------+
       Total:                     1142    220       0      
                                                           
    C:/ti/TivaWare_C_Series-2.1.4.178/sensorlib/ccs/Debug/sensorlib.lib
       i2cm_drv.obj               1414    0         0      
       mpu9150.obj                870     32        0      
       bmp180.obj                 820     0         0      
    +--+--------------------------+-------+---------+---------+
       Total:                     3104    32        0      
                                                           
    G:\Code\ccsv7\tools\compiler\ti-cgt-arm_16.9.4.LTS\lib\rtsv7M4_T_le_v4SPD16_eabi.lib
       e_powf.obj                 1416    24        0      
       strtod.obj                 572     152       0      
       fd_add_t2.obj              438     0         0      
       fd_div_t2.obj              310     0         0      
       ctype.obj                  0       257       0      
       fd_mul_t2.obj              252     0         0      
       s_scalbnf.obj              212     0         0      
       memcpy_t2.obj              156     0         0      
       fd_cmp_t2.obj              134     0         0      
       memset_t2.obj              122     0         0      
       autoinit.obj               112     0         0      
       fd_tos_t2.obj              110     0         0      
       copy_decompress_lzss.obj   104     0         0      
       exit.obj                   84      0         12     
       boot.obj                   84      0         0      
       fs_toull_t2.obj            80      0         0      
       cpy_tbl.obj                76      0         0      
       u_divt2.obj                64      0         0      
       e_sqrtf.obj                40      0         0      
       _lock.obj                  20      0         8      
       args_main.obj              24      0         0      
       strcpy.obj                 20      0         0      
       strlen.obj                 20      0         0      
       s_copysignf.obj            18      0         0      
       copy_decompress_none.obj   14      0         0      
       copy_zero_init.obj         12      0         0      
       errno.obj                  0       0         4      
       pre_init.obj               4       0         0      
       stkdepth_vars.obj          0       0         4      
       i_div0.obj                 2       0         0      
       mpu_init.obj               2       0         0      
       startup.obj                2       0         0      
    +--+--------------------------+-------+---------+---------+
       Total:                     4504    433       28     
                                                           
       Stack:                     0       0         1024   
       Linker Generated:          0       58        0      
    +--+--------------------------+-------+---------+---------+
       Grand Total:               12810   1399      2738   


LINKER GENERATED COPY TABLES

__TI_cinit_table @ 00003788 records: 2, size/record: 8, table size: 16
	.data: load addr=00003758, load size=00000016 bytes, run addr=20000a80, run size=00000038 bytes, compression=lzss
	.bss: load addr=00003780, load size=00000008 bytes, run addr=20000000, run size=0000067d bytes, compression=zero_init


LINKER GENERATED HANDLER TABLE

__TI_handler_table @ 00003770 records: 3, size/record: 4, table size: 12
	index: 0, handler: __TI_decompress_lzss
	index: 1, handler: __TI_decompress_none
	index: 2, handler: __TI_zero_init


GLOBAL SYMBOLS: SORTED ALPHABETICALLY BY Name 

address   name                           
-------   ----                           
000033c1  BMP180AppCallback              
00002bc9  BMP180DataRead                 
00002489  BMP180DataTemperatureGetFloat  
000033fd  BMP180DataTemperatureGetRaw    
00003409  BMP180I2CIntHandler            
00002c21  BMP180Init                     
00002d71  C$$EXIT                        
000029e1  ConfigureUART                  
00003215  GPIODirModeSet                 
0000185f  GPIOPadConfigSet               
00003389  GPIOPinTypeI2CSCL              
0000345b  GPIOPinWrite                   
00002379  I2CMCommand                    
00003183  I2CMInit                       
00001ca1  I2CMIntHandler                 
00002605  I2CMReadModifyWrite8           
0000346d  I2CMasterControl               
00003471  I2CMasterDataGet               
00003475  I2CMasterDataPut               
00003439  I2CMasterEnable                
00002e65  I2CMasterInitExpClk            
00003443  I2CMasterIntClear              
0000344b  I2CMasterIntEnableEx           
00003453  I2CMasterSlaveAddrSet          
00002841  IntDisable                     
000028a9  IntEnable                      
00002a45  IntIsEnabled                   
00003415  IntTrigger                     
00003421  MPU9150Callback                
0000250d  MPU9150DataAccelGetFloat       
0000314d  MPU9150DataMagnetoGetRaw       
00002b09  MPU9150DataRead                
000027d5  MPU9150Init                    
00002c75  MPU9150ReadModifyWrite         
00003291  PWMGenConfigure                
000033d1  PWMGenPeriodSet                
00003115  RGBBlinkIntHandler             
0000267d  RGBBlinkRateSet                
0000225d  RGBColorSet                    
00002911  RGBDisable                     
00001e69  RGBEnable                      
00001aa1  RGBInit                        
00003339  RGBIntensitySet                
00003461  ResetISR                       
UNDEFED   SHT$$INIT_ARRAY$$Base          
UNDEFED   SHT$$INIT_ARRAY$$Limit         
00001991  SysCtlClockGet                 
000031b9  SysTickIntHandler              
00003467  UARTClockSourceSet             
000031e9  UARTFlushRx                    
000030d9  UARTFlushTx                    
00002fd5  UARTPeek                       
00001f29  UARTStdioConfig                
000015c9  UARTStdioIntHandler            
00002cc9  UARTgets                       
000032ed  UARTprintf                     
00001095  UARTvprintf                    
00001fd9  UARTwrite                      
20000a80  __STACK_END                    
00000400  __STACK_SIZE                   
20000a80  __STACK_TOP                    
00003788  __TI_CINIT_Base                
00003798  __TI_CINIT_Limit               
00003770  __TI_Handler_Table_Base        
0000377c  __TI_Handler_Table_Limit       
000026f5  __TI_auto_init                 
20000a98  __TI_cleanup_ptr               
00002979  __TI_decompress_lzss           
000033ef  __TI_decompress_none           
20000a9c  __TI_dtors_ptr                 
20000aa0  __TI_enable_exit_profile_output
ffffffff  __TI_pprof_out_hndl            
ffffffff  __TI_prof_data_size            
ffffffff  __TI_prof_data_start           
00000000  __TI_static_base__             
0000342d  __TI_zero_init                 
00002401  __aeabi_cdcmpeq                
00002401  __aeabi_cdcmple                
00002765  __aeabi_d2f                    
00001289  __aeabi_dadd                   
00001729  __aeabi_ddiv                   
00001ba5  __aeabi_dmul                   
0000127f  __aeabi_dsub                   
00002e15  __aeabi_f2ulz                  
000027d3  __aeabi_idiv0                  
00002589  __aeabi_memclr                 
00002589  __aeabi_memclr4                
00002589  __aeabi_memclr8                
00002129  __aeabi_memcpy                 
00002129  __aeabi_memcpy4                
00002129  __aeabi_memcpy8                
0000258b  __aeabi_memset                 
0000258b  __aeabi_memset4                
0000258b  __aeabi_memset8                
0000305b  __aeabi_uidiv                  
0000305b  __aeabi_uidivmod               
ffffffff  __binit__                      
ffffffff  __c_args__                     
00002bc7  __mpu_init                     
20000680  __stack                        
00003321  _args_main                     
00002d1d  _c_int00                       
00003480  _ctypes_                       
20000aa4  _lock                          
0000335b  _nop                           
00003353  _register_lock                 
0000334d  _register_unlock               
00002fd3  _system_post_cinit             
00003479  _system_pre_init               
20000aa8  _unlock                        
00002d75  abort                          
ffffffff  binit                          
00002081  comenzi                        
00002eb1  copy_in                        
000033ad  copysignf                      
20000ab0  errno                          
00002d7d  exit                           
2000067c  g_bMPU9150Done                 
00000000  g_pfnVectors                   
20000660  g_pui32Colors                  
20000610  g_sBMP180Inst                  
20000400  g_sI2CInst                     
20000678  g_vui8DataFlag                 
00001d95  ldexpf                         
000007f5  main                           
20000ab4  main_func_sp                   
00002129  memcpy                         
00002591  memset                         
0000026d  powf                           
200005a4  sMPU9150                       
00001d95  scalbnf                        
00003269  sqrtf                          
00003361  strcpy                         
00003375  strlen                         
00000c61  strtod                         
00000c61  strtold                        


GLOBAL SYMBOLS: SORTED BY Symbol Address 

address   name                           
-------   ----                           
00000000  __TI_static_base__             
00000000  g_pfnVectors                   
0000026d  powf                           
00000400  __STACK_SIZE                   
000007f5  main                           
00000c61  strtod                         
00000c61  strtold                        
00001095  UARTvprintf                    
0000127f  __aeabi_dsub                   
00001289  __aeabi_dadd                   
000015c9  UARTStdioIntHandler            
00001729  __aeabi_ddiv                   
0000185f  GPIOPadConfigSet               
00001991  SysCtlClockGet                 
00001aa1  RGBInit                        
00001ba5  __aeabi_dmul                   
00001ca1  I2CMIntHandler                 
00001d95  ldexpf                         
00001d95  scalbnf                        
00001e69  RGBEnable                      
00001f29  UARTStdioConfig                
00001fd9  UARTwrite                      
00002081  comenzi                        
00002129  __aeabi_memcpy                 
00002129  __aeabi_memcpy4                
00002129  __aeabi_memcpy8                
00002129  memcpy                         
0000225d  RGBColorSet                    
00002379  I2CMCommand                    
00002401  __aeabi_cdcmpeq                
00002401  __aeabi_cdcmple                
00002489  BMP180DataTemperatureGetFloat  
0000250d  MPU9150DataAccelGetFloat       
00002589  __aeabi_memclr                 
00002589  __aeabi_memclr4                
00002589  __aeabi_memclr8                
0000258b  __aeabi_memset                 
0000258b  __aeabi_memset4                
0000258b  __aeabi_memset8                
00002591  memset                         
00002605  I2CMReadModifyWrite8           
0000267d  RGBBlinkRateSet                
000026f5  __TI_auto_init                 
00002765  __aeabi_d2f                    
000027d3  __aeabi_idiv0                  
000027d5  MPU9150Init                    
00002841  IntDisable                     
000028a9  IntEnable                      
00002911  RGBDisable                     
00002979  __TI_decompress_lzss           
000029e1  ConfigureUART                  
00002a45  IntIsEnabled                   
00002b09  MPU9150DataRead                
00002bc7  __mpu_init                     
00002bc9  BMP180DataRead                 
00002c21  BMP180Init                     
00002c75  MPU9150ReadModifyWrite         
00002cc9  UARTgets                       
00002d1d  _c_int00                       
00002d71  C$$EXIT                        
00002d75  abort                          
00002d7d  exit                           
00002e15  __aeabi_f2ulz                  
00002e65  I2CMasterInitExpClk            
00002eb1  copy_in                        
00002fd3  _system_post_cinit             
00002fd5  UARTPeek                       
0000305b  __aeabi_uidiv                  
0000305b  __aeabi_uidivmod               
000030d9  UARTFlushTx                    
00003115  RGBBlinkIntHandler             
0000314d  MPU9150DataMagnetoGetRaw       
00003183  I2CMInit                       
000031b9  SysTickIntHandler              
000031e9  UARTFlushRx                    
00003215  GPIODirModeSet                 
00003269  sqrtf                          
00003291  PWMGenConfigure                
000032ed  UARTprintf                     
00003321  _args_main                     
00003339  RGBIntensitySet                
0000334d  _register_unlock               
00003353  _register_lock                 
0000335b  _nop                           
00003361  strcpy                         
00003375  strlen                         
00003389  GPIOPinTypeI2CSCL              
000033ad  copysignf                      
000033c1  BMP180AppCallback              
000033d1  PWMGenPeriodSet                
000033ef  __TI_decompress_none           
000033fd  BMP180DataTemperatureGetRaw    
00003409  BMP180I2CIntHandler            
00003415  IntTrigger                     
00003421  MPU9150Callback                
0000342d  __TI_zero_init                 
00003439  I2CMasterEnable                
00003443  I2CMasterIntClear              
0000344b  I2CMasterIntEnableEx           
00003453  I2CMasterSlaveAddrSet          
0000345b  GPIOPinWrite                   
00003461  ResetISR                       
00003467  UARTClockSourceSet             
0000346d  I2CMasterControl               
00003471  I2CMasterDataGet               
00003475  I2CMasterDataPut               
00003479  _system_pre_init               
00003480  _ctypes_                       
00003770  __TI_Handler_Table_Base        
0000377c  __TI_Handler_Table_Limit       
00003788  __TI_CINIT_Base                
00003798  __TI_CINIT_Limit               
20000400  g_sI2CInst                     
200005a4  sMPU9150                       
20000610  g_sBMP180Inst                  
20000660  g_pui32Colors                  
20000678  g_vui8DataFlag                 
2000067c  g_bMPU9150Done                 
20000680  __stack                        
20000a80  __STACK_END                    
20000a80  __STACK_TOP                    
20000a98  __TI_cleanup_ptr               
20000a9c  __TI_dtors_ptr                 
20000aa0  __TI_enable_exit_profile_output
20000aa4  _lock                          
20000aa8  _unlock                        
20000ab0  errno                          
20000ab4  main_func_sp                   
ffffffff  __TI_pprof_out_hndl            
ffffffff  __TI_prof_data_size            
ffffffff  __TI_prof_data_start           
ffffffff  __binit__                      
ffffffff  __c_args__                     
ffffffff  binit                          
UNDEFED   SHT$$INIT_ARRAY$$Base          
UNDEFED   SHT$$INIT_ARRAY$$Limit         

[136 symbols]
